:100000000C943E000C9448000C9448000C9448005A
:100010000C9448000C9448000C9448000C94480040
:100020000C9448000C9448000C9448000C94480030
:100030000C9448000C9448000C9448000C94480020
:100040000C9448000C9448000C9448000C94480010
:100050000C9448000C9448000C9448000C94480000
:100060000C9448000C9448000C9448000C944800F0
:100070000C9448000C9448000C94480011241FBEB6
:10008000CFEFCDBFDFE3DEBF0E944A000C946400D7
:100090000C94000088ED84BF10926100059A0D9ABF
:1000A0002FEF81E19AE7215080409040E1F700C0B6
:1000B00000000D982FEF88E09DE321508040904094
:0C00C000E1F700C00000EBCFF894FFCF88
:00000001FF
